:100000000206B4C0E0C0D075D000C000781A06E681
:1000100018700106C2CFD000D0D0D0E03202190053
:020020000000DE
:0300230002074091
:10002B00020003E4F52DF5347535FF753625F537EC
:10003B00F538F539F53A1207BB7BFF7A08790512CB
:10004B0008977BFF7A087918120897C297D290E429
:10005B007819F608F6C3781AE6942818E694004047
:10006B00F4D2977BFF7A08792B120897120952C2A8
:10007B00FFE4F5A375ECFF1208BCD3EF9400EE94EC
:10008B0000400543340880035334F77819E6FE0823
:10009B00E6FF65387003EE6537600C8E378F3805D9
:1000AB003AE53A70020539C3EF9450EE94004006DE
:1000BB00E47819F608F6C3E53A94C8E5399400409C
:1000CB000F753900753AC8D290D2975334CF801E32
:1000DB00C3E53A9464E53994004007D2975334EF63
:1000EB00800CE53430E407C29730E502C2908534CA
:1000FB003530FF80C2FF85A321E52DB40E004003F0
:10010B00020324900115F828287302013F02017E97
:10011B000201870201990201AC0202A3020324022D
:10012B00030002030202031502021F02022902024C
:10013B002F020263E52124AB601B24B2601D146007
:10014B002014602924FB601F2450600302007F757C
:10015B002D0102007F752D0402007F752D09020011
:10016B007F8536A302007F752D0802007F8534A39F
:10017B0002031E85212E752D0202007F85212FE59E
:10018B002F7005F52D02007F752D0302007FAF2127
:10019B0012060F152FE52F600302007FF52D0200CD
:1001AB007F85212E1208BC8E308F31D3EF9400EE59
:1001BB0094004058D3E5319408E53094004006751F
:1001CB003000753108AF31EFF5A3E4F522E52E646D
:1001DB000270338F22F532F533F521E521C39522D9
:1001EB00501E12043974242521F8A60774242521E6
:1001FB00F8E67E002533FF7532008F33052180DB57
:10020B00752D0A02007F752D0502007FE4F5A3F51D
:10021B002D02007FE522F4F5A3E4F5238034752D40
:10022B000C02007FE521B4060302031EE521B4187E
:10023B001BE4F521E521C39522500E74242521F8EA
:10024B00E6FF1208DF052180EB02031E8524A37550
:10025B002301752D0D02007FE521B4181BE4F52158
:10026B00E521C39522500E74242521F8E6FF1208D0
:10027B00DF052180EB02031EE523C39522500EAF51
:10028B0023052374242FF8E6F5A302007FE533F44E
:10029B00F5A3752D0B02007FE521B4181AE4F521A7
:1002AB00E521C39522500E74242521F8E6FF120890
:1002BB00DF052180EB805CD3E5319400E5309400C1
:1002CB0040311204398F218521A3AF2205227424DA
:1002DB002FF8A621E522C394094003752208E531C6
:1002EB00153170021530144530600302007FF52D77
:1002FB0002007F801E801C5334F8E52154374234B2
:10030B00E4F539F53AF52D02007FAF211205458F43
:10031B00368FA3E4F52D02007FE4F52D02007FE775
:10032B0009F608DFFA8046E709F208DFFA803E8813
:10033B00828C83E709F0A3DFFA8032E309F608DF4A
:10034B00FA8078E309F208DFFA807088828C83E305
:10035B0009F0A3DFFA806489828A83E0A3F608DFC1
:10036B00FA805889828A83E0A3F208DFFA804C80F6
:10037B00D280FA80C680D4806980F280338010806E
:10038B00A680EA809A80A880DA80E280CA803389CE
:10039B00828A83ECFAE493A3C8C582C8CCC583CC0C
:1003AB00F0A3C8C582C8CCC583CCDFE9DEE7800DDE
:1003BB0089828A83E493A3F608DFF9ECFAA9F0EDBE
:1003CB00FB2289828A83ECFAE0A3C8C582C8CCC51C
:1003DB0083CCF0A3C8C582C8CCC583CCDFEADEE8EA
:1003EB0080DB89828A83E493A3F208DFF980CC88CF
:1003FB00F0EF60010E4E60C388F0ED2402B40400F0
:10040B0050B9F582EB2402B4040050AF232345828C
:10041B002390037A73BB010689828A83E022500200
:10042B00E722BBFE02E32289828A83E49322D379FB
:10043B0012E778169619E71896500F9001DAE0FF3D
:10044B009001D9E09F50037FFF229001DAE0FF90EB
:10045B0001D9E0FED39F405DA3E004F074DB2FF5E0
:10046B0082E43401F583E0F53B9001DAE0FFB50659
:10047B000AE49001D9F0A3F002053CEFD3940F509E
:10048B000302053C9001D9E0FFA3E0FEEF9E900133
:10049B00D9F0F58275830074DB2EF9E43401FA7B15
:1004AB000178DB7C017D017E00AF821203FAE490C0
:1004BB0001DAF0807CE49001D9F0A3F07811E6FE2C
:1004CB0008E6FFD3781696EE1896405A0806E618FB
:1004DB008604700106142401F58274003CF583E058
:1004EB00F53B7815E6FC08E6FDB5070CECB5060800
:1004FB00E47811F608F6802AD3ED946AEC94004068
:10050B00307812E69DFF18E69CFEF608EFF67401B4
:10051B002DF974003CFA7B0178017C007D011203FC
:10052B00FAE478158008E47815F608F67811F608E1
:10053B00F6D292D294D293AF3B228F3C538EF4E5FA
:10054B003CC39425404DC2CA75B28375CB9C75CA0A
:10055B004FD2CAE53C24C8601624ED601724DB603B
:10056B001824DA601924B5601A24BC701E801F751C
:10057B008DB8806D758DCB8068758D968056758D19
:10058B00B08051758D2B438E088056753C25758D2B
:10059B0096804EC2CA75B28075CB3C75CAB0D2CAB2
:1005AB00E53C24FE601924FE601D24FB601E24F72D
:1005BB00601F24ED602324247021758D96800375B4
:1005CB008DCB438E02801A758D6A8015758D608078
:1005DB0003758DB0438E0180088003753C25758DA6
:1005EB00A0D200D202C201E47811F608F69001D92C
:1005FB00F008F608F67817F608F67815F608F6A35D
:10060B00F0AF3C228F3FD37818E6940018E69400A5
:10061B004059D2017817E6FE08E6FF7813E6FC088E
:10062B00E6FDD39FEC9E500AE47817F608F6781394
:10063B008034C3EF944BEE9400402EED78189679EE
:10064B0014F7EC189619F77813E6FE08E6FF7818FE
:10065B00E62442F9E43401FA7B0178427C017D0106
:10066B001203FAE47817F608F6C201C37814E6947D
:10067B009518E6940040107818E6184670943002EE
:10068B00F6C202D29980F078130806E61886067037
:10069B000106142442F58274013EF583E53FF030E8
:1006AB000204C202D299AF3F22787FE4F6D8FD75DF
:1006BB00813F0206FB02002EE493A3F8E493A340D0
:1006CB0003F68001F208DFF48029E493A3F85407C2
:1006DB00240CC8C333C4540F4420C8834004F456BD
:1006EB00800146F6DFE4800B0102040810204080F5
:1006FB0090001DE47E019360BCA3FF543F30E509DD
:10070B00541FFEE493A360010ECF54C025E060A8F4
:10071B0040B8E493A3FAE493A3F8E493A3C8C58287
:10072B00C8CAC583CAF0A3C8C582C8CAC583CADFF5
:10073B00E9DEE780BEC0E0C083C082C0D075D008C0
:10074B0030982FC298C37812E6943F18E694015064
:10075B00150806E618860E700106142401F582743E
:10076B00003EF5838009C292C294C293900000E5CB
:10077B0099F0309932C29920012BD37914E778186C
:10078B009619E7189640180806E618860E700106AB
:10079B00142442F58274013EF583E0F5998002D270
:1007AB0002D2008002D202D0D0D082D083D0E032ED
:1007BB0053D9BFE4F5A8F5B8F5E6F5F675E477D2AD
:1007CB009712094B75D90275EBFF75ECFF12093BBC
:1007DB001208F9120912120871E4F53B12092905E6
:1007EB003BE53BC3946440F4D2AFE4F53B120929DB
:1007FB00053BE53BC3946440F422202020202020BD
:10080B00202020202020202020200D0A004E4F41A8
:10081B00412033333120537461727475700D0A00AB
:10082B004E4F414120333331204C6F6F700D0A0016
:10083B008F3EE53ED3947F40037F0022E53EB40A12
:10084B00057F0D12060FE53EC394205011E53E24A3
:10085B00F824FD500924FE600580007F0022AF3E86
:10086B0012060FAF3E22C299C28EC2AB759810D240
:10087B009C7F25120545758BFF53890F438920C239
:10088B0099C298D2ACD2BCD299D28E228B3B8A3CE5
:10089B00893DAB3BAA3CA93D1204206013053DE505
:1008AB003D7002053C14F9120420FF12083B80E254
:1008BB00229001DAE0FF9001D9E0C39FFFE494009E
:1008CB00FEC37912E7781696FD19E71896CD2FFF20
:1008DB00ED3EFE229001D9E0C3941D5010E0FE04C2
:1008EB00F074DB2EF582E43401F583EFF02275A46E
:1008FB005475A5F475F1FF75F2FFE4F5D475D5FFCA
:10090B0075E10B75E24022E4F5C8538ECF75CB9E93
:10091B0075CA5874FFF5CDF5CCD2ADD2CA22E4FF1F
:10092B00FE75ECFF0FBF00010EBE01F5BFF4F22206
:10093B0075A20B75A10775F804D2F9D2F8C2FF2284
:0E094B00E4F5A975B28322E47811F608F622CD
:00000001FF
